:030000000219FDE5
:03000B000200A848
:03002B0002015A75
:03005B000202EBB3
:030073000202D8AE
:1000800002030406080C10182030406080040608A3
:100090000C10182030406080A0C00003070F1F051F
:1000A000050D050305030302C2AFC0D0C0E0206206
:1000B00014E5256009E473E525F4F58AD262D0E001
:1000C000D0D0D2AF3285268AC262E526F4602F30C6
:1000D000682520720DD0E0D0D0C2B1C287C281D2D3
:1000E000AF32C2B1C287C281206F0C206509740A89
:1000F000D5E0FDE57B4280D0E0D0D0D2AF32758A2A
:1001000000C28DD26201F701B7306805206502D2C6
:10011000B101B7306805206502D28701B7306805A4
:10012000206502D28101B7C28230680A2065077457
:1001300008D5E0FDD2B101B7C28630680A20650754
:100140007408D5E0FDD28701B7C28030680A206507
:10015000077408D5E0FDD28101B7C2AFC2AD53E646
:10016000EFC0D0C0E0D2D3D2AFC2CEE52A60072024
:10017000744F152A21C17800790020742EE5803053
:100180007E01F430E50278FF53DACF207E0343DAB4
:1001900020307E0343DA10C2D8C271E580307E0180
:1001A000F430E50279FFC3E89970CB306103752A1A
:1001B00018207403752A18885CD270E86003755F94
:1001C0000020740DE52B6004152B21D143DA01C208
:1001D000D82070024144A85C206102C270207431B2
:1001E000C3E894F0400374F0F8E8C4540F28F87999
:1001F00084B703024111C313C3138721200802C32C
:1002000013200A06C3C898F8411128F8500374FF58
:10021000F8C3E895655003E565F88822E52D540696
:100220006022206B1FE536C333C333F8E564C31384
:10023000C313F9C3952240028922E82522F52250F2
:10024000037522FF852224A824C3E524956140027A
:10025000A8618825E56670024188C3E8AA669A50BD
:1002600003E8FAE4F9EAC333FBE568F45B29400DDF
:100270002567F8E56760021567400B41880AC3E50A
:10028000679A5002056778FF8826C26FC3E52694F7
:10029000F84002D26F20CF0AD0E0D0D043E610D28F
:1002A000AD32C2CF053A7801E52A600530740215F7
:1002B0002AC3E55C94014005755F0041CE7560007E
:1002C000756900E55F2401F55F5003755FFFD0E0BD
:1002D000D0D043E610D2AD32C2AF53E67F7592FA6A
:1002E0007593FFC260759104D2AF32C2AF53E6EF8F
:1002F000C2ADC0D0C0E0C0F0D2D3D2AFA8FBA9FC41
:10030000C2D8307102615253DACF207E0343DA1033
:10031000307E0343DA20D271E580307E01F420E59F
:1003200002612988278928A17F53DACF207E0343E1
:10033000DA20307E0343DA10C2D8C271307402A1D1
:100340006B7800E580307E01F430E502A16B885CBB
:10035000A15353DACF207E0343DA20307E0343DA01
:1003600010C271206102812B53DACF207E0343DA61
:1003700010307E0343DA20C2D8D27188578958C31F
:10038000E89555F8E99556F97B007E087A00C3E8B0
:10039000948CE994005005755B00811D882178A23A
:1003A000E6A8216055C3E894C8E994005008E4D257
:1003B000E4FB7A0A61F8C3E89468E994015008E420
:1003C000D2E3FB7A0F61F8C3E894D0E994025008B5
:1003D000E4D2E2FB7A1E61F8C3E894A0E9940550E8
:1003E00008E4D2E1FB7A3C61F8C3E89498E9940808
:1003F0005008E4D2E0FB7A787E00C3E89559FCE926
:10040000955AFD30E70AECF42401FCEDF43400FDCC
:10041000755B00C3EC9AED9E5003755B01885989AA
:100420005A8557558558567802A153C3E89527F841
:10043000E99528F9307C02A137307B02A137307A68
:1004400002A130207502814EE9FDE8FC816DE9C30F
:1004500013F9E813F8307902A130E9C313F9E8136E
:10046000F8307802A130E9C313FDE813FC20612CB9
:0F047000C3EC941CED940240028184ED701EC316
:10047F00EC94C850180529E52970021529C3E52900
:10048F00940A5002A16B755C00D270A16BE52960D4
:10049F000215297888E6F97400207F087896B90349
:1004AF0002789EE624FAFEE43400FFC3EC9EFCEDD6
:1004BF009FFD9208B90310A2085007207609D27643
:1004CF0081D6307602C276A2085016B9030DECF42D
:1004DF002401FCEDF43400FD0204F078007900A152
:1004EF0037B90315EC33FCED33FDC3EC940AFCED87
:1004FF009400FD50047C007D00C3EC94FFED94004C
:10050F00400678FF7900A137EC8572F0A4C5F0A200
:10051F00F733F87900400302055378FF790002059D
:10052F0053E9C313F9E813F8307C0EE9600278FF42
:10053F00C3E81338F8E43400F9C3E894FFE99400F2
:10054F00400278FF885CD270206102A16B741FF4A7
:10055F00552F4BF52FC274EB7002D274752A1830D9
:10056F007403752A0A306102A17F20740353DAFEE7
:10057F00207403752B06D0F0D0E0D0D0D2AD43E677
:10058F00103279010205AF79030205AF790A02052E
:10059F00AF791E0205AF79640205AF79C80205AFC6
:1005AF007817E4D5E0FDD8FAD9F6227A147B7802D1
:1005BF0005D67A107B8C0205D67A0D7BB40205D650
:1005CF007A0B7BC80205D6E573D5E001227902E4E8
:1005DF00C286D5E0FDD287D5E0FDC287D5E0FDD23A
:1005EF0086D5E0FDE920E002D2B130E002D281E50C
:1005FF0073D5E0FDE920E002C2B130E002C28174A0
:10060F0096D5E0FDD9C9EAF8D5E0FDD8FBDBB8C235
:10061F008622C37C007D0075F00005F0EA33FAEB0B
:10062F0033FB50F6EB13FBEA13FAC3E9FFE8FEE8DE
:10063F009AF8E99BF95004EFF9EEF8B3EC33FCEDBF
:10064F0033FDD5F0DFEDF9ECF822E889F08A20D2FE
:10065F00D4F8A9F07B0030F70B7BFFF42401F8E905
:10066F00F43400F9E88520F0A4ADF0F8E98520F026
:10067F00A4AFF0FEED2EF974003FFA7C04C3EA1329
:10068F00FAE913F9E813F8DCF48BF030F70AE8F421
:10069F002401F8E9F43400F9E889F0C2D4F8A9F09C
:1006AF002222C3E54113F9E54013F8C3E54498F856
:1006BF00E54599F9500CC3E89480E994FF40160280
:1006CF0006E8C3E8947FE9940050030206E8787FB8
:1006DF0079000206E8788079FF8849894A22E5493E
:1006EF002546F8E54A3547F9854A20E4300701F4F5
:1006FF003548FA30E709C3EA94F04015020726C3DC
:10070F00EA940F500302072678FF79FF7A0F02074A
:10071F0026780079007AF0C3E5249561500AC374F6
:10072F00019524500B020744E54A20E70E020744C7
:10073F00E54A30E706884689478A482278A5E6FACF
:10074F00C3E54933F8E54A33F9D159E930E70BC32B
:10075F00E89480E994FF4013E17EC3E8947FE99425
:10076F00005002E17E787F7900E17E788079FFE8A2
:10077F0020E715C3E52398F84009C3E89401400327
:10078F000207A578010207A5E8F424012523F84004
:10079F00030207A578FF884B2278A6E6FAA847A997
:1007AF0048D159E930E70CC3E89401E994FF4016AA
:1007BF000207D9C3E894FFE9940050030207D978E0
:1007CF00FF79000207D9780179FFE920E715C3E522
:1007DF004B98F84009C3E8940140030208007801E0
:1007EF00020800E8F42401254BF8400302080078C2
:1007FF00FF88242278FF20692879A1E76023E5414B
:10080F00601F74FF8541F0848539F0306A0375F0FD
:10081F0005A4F8C5F0600278FFC3E895645002A8FC
:10082F0064886322C3E5409440E5419401E5635039
:10083F0003140144046002F5632202084C2275E898
:10084F0090227883E6FF30EDF9A8BDA9BE0570C3ED
:10085F00E57094084052757000E9FA79A0E760449A
:0E086F00EA7007E571601B020885C3E8957109
:10087D006010E5715006600C140208910460F902D5
:10088D000891E571F571C394A8401B7561C0C394BF
:10089D00054013756180C39405400B756140C39489
:1008AD0005400375610075BB0622E561F460020524
:1008BD0061E570B4070375BB1E22743279A787F00A
:1008CD00A4C5F0A2F733F8C3E895614002A861888A
:1008DD00228824882588268864227540007541F079
:1008ED0022C2AF75C820A8CCA9CDAA3A30CF010A33
:1008FD0075C824D2AFAB3BAC3C883B893CC3E89B6D
:10090D00F8E99C206908F930660221FF2159AD3DB7
:10091D008A3DF9EA9DFA600678FF79FF213EAE3EE9
:10092D00AF3F8B3E8C3FA83BA93CC3E89EF8E99FA7
:10093D00F9C3E54113FBE54013FAE82AF540E93B1D
:10094D00F54150067540FF7541FF21A6AA40AB4108
:10095D00AC40AD417E047F02C3EB9404400D1E1FDD
:10096D00C3EB94084005206A021E1FC3ED13FDEC76
:10097D0013FCDEF7C3EA9CFAEB9DFBEF6009C3E9BC
:10098D0013F9E813F8DFF7EA28FAEB39FB8A408B05
:10099D004150067BFF8B408B41C3EB94025002D23A
:1009AD00663069047F0321D17892E6FFC3E5379461
:1009BD008240110FC3E53794A040010FC3EF940699
:1009CD0040027F057E02E541C4540FF9E541C45450
:1009DD00F0F8E540C4540F28F8C3E89EFAE99400F6
:1009ED00FB4009C3EA9402EB940050047A02E4FB45
:1009FD00414BAA40AB41EBC4FEEAC4540F4EFCC3BD
:100A0D00EA9CFAEB9400FBC3E813C313F8EA28FA47
:100A1D00EB3400FB8A408B41C3EB94024002C2666B
:100A2D007802EBC4FE7B00EAC4540F4EFAC3EA9879
:100A3D00FA4005C3940250027A027892E6FF3060C4
:100A4D0002414B855192855293D26043E680C3E4B7
:100A5D009AF8E49BF930660241D7E8FAE9FBD3E94D
:100A6D0013FDE813FC88518952C3EF94036038EFEE
:100A7D0020E00DE82CF8E93DF9ECFAEDFB020AA0B7
:100A8D00E828F8E939F9C3E82402F8E93400F97ADD
:100A9D00FE7BFFC3EF9403400E8A538B54884D8920
:100AAD004E8C4F8D50610B885389548A4D8B4E8CD3
:100ABD004F8D503069127553F07554FF754FF075A9
:100ACD0050FF7551F07552FF610BE8FAD3E813FC36
:100ADD008851C3EF94036020EF20E007E82CF8EC79
:100AED00FA41F7E8282402F87AFEC3EF9403400890
:100AFD008A53884D8C4F610B88538A4D8C4FE56816
:100B0D00C3335002646BF5683060026115753402B1
:100B1D00D26043E680E52D54066034A840A941C358
:100B2D00E913F9E813F8C3E913F9E813F830690488
:100B3D00E92440F9C2AF53E67F759100C3E498F5FF
:100B4D0094E499F595759104D26043E680D2AF2275
:100B5D00D264754300752000306C03752040020B84
:100B6D007CD264754300752040306C03752000788D
:100B7D00017901206620E52D54066002C2647914C6
:100B8D00E541C313700104F8C39414400278143086
:100B9D006904781B791B206010E543600C306903F4
:100BAD00D53404D26D8126711D0543E59B5440B5A6
:100BBD002002811030690908C3E89940011861A32A
:100BCD0020640A08C3E8994002617C61A3C264C233
:100BDD00AF53E67F7591003066127594007595F8E8
:100BED00759104D26043E680D2AF617CE5417EFF12
:100BFD00C3334005C3334001FEC3E49E759400F535
:100C0D009561EDC3E53394015002617C306402615E
:100C1D007CD802812461A3C26DC2AF53E67F75916A
:100C2D0000855394855495759104854D92854E9309
:100C3D00D26043E680D2AFE52D54066008206A02EB
:100C4D000533020C62306D0D206C0A20640715818E
:100C5D0015810215402278003064027801E5377560
:0F0C6D00F007A4F9E5F028F5F0E9A2F013A2F1E1
:100C7C0013A2F213F537C394785003753778C3E594
:100C8C003795384008D265C2B1C287C28130600244
:100C9C008199854F92855093D26043E68022207DC6
:100CAC0016C2AF754202C286D282306202D281D2A3
:100CBC00AF759F02020E9AC2AF754202C286D280F5
:100CCC00306202D2B1D2AF759F02020E9A307243DB
:100CDC00207D20C2AF754203900138757B40C281E4
:100CEC00C280306204D28781F7D286D2AF759F035F
:100CFC00020E9AC2AF754203900138757B40C2B1A7
:100D0C00C282306204D287A117D286D2AF759F01FE
:100D1C00020E9A207D17C2AF754203900113C28157
:100D2C00306202D287D2AF759F03020E9AC2AF75A2
:100D3C004203900113C2B1306202D287D2AF759FC9
:100D4C0001020E9A207D16C2AF754204C282D28077
:100D5C00306202D287D2AF759F01020E9AC2AF7574
:100D6C004204C280D282306202D287D2AF759F0316
:100D7C00020E9A307243207D20C2AF75420590015D
:100D8C0027757B04C287C286306204D2B1A19DD282
:100D9C0082D2AF759F02020E9AC2AF7542059001C6
:100DAC0049757B01C287C286306204D281A1BDD253
:100DBC0080D2AF759F02020E9A207D17C2AF75428A
:100DCC0005900109C287306202D2B1D2AF759F0281
:100DDC00020E9AC2AF75420590011DC2873062EBBC
:100DEC00D281D2AF759F02020E9A207D16C2AF75CA
:100DFC004206C280D286306202D2B1D2AF759F0356
:100E0C00020E9AC2AF754206C282D286306202D2FC
:100E1C0081D2AF759F01020E9A307244207D20C2A0
:100E2C00AF754201900149757B01C2B1C28230623B
:100E3C0004D281C143D280D2AF759F01020E9AC2F7
:100E4C00AF754201900127757B04C281C28030626C
:100E5C0005D2B1020E64D282D2AF759F03020E9AF4
:100E6C00207D17C2AF75420190011DC2B1306202E4
:100E7C00D281D2AF759F01020E9AC2AF754201901A
:100E8C000109C281306202D2B1D2AF759F03C26533
:100E9C0022900107757B00C2B1C287C281C282C297
:100EAC0086C280C26222788076FF0876FF0876FFC1
:100EBC000876FF0876030876040876090876030896
:100ECC007601087601788C76010876FF0876FF08A3
:100EDC0076FF0876FF0876FF0876030876FF08761B
:100EEC00FF0876FF0876250876D00876FA0876FA99
:100EFC000876040876FF08760108760008767A08EA
:100F0C0076FF0876010876010876000876030876E5
:100F1C0000227887E6FFC272BF0302D2727888E69D
:100F2C00C394036008C27DE630E102D27DC27E78B4
:100F3C0089E630E102D27EC3EF94026008758E011F
:100F4C00D273020F56758E00C273227880E614900D
:100F5C0000809378A5F67881E6149000809378A6AB
:100F6C00F67886E61490008D9378A7F67886E6F5E9
:100F7C0039C394025003753902789CE67538FFB476
:100F8C0002037538A0B4030375388278A3E6149075
:100F9C00009A93F566D19D22227896E6FA7897E628
:100FAC00FB7888E6B40305C3EB940EFB307F047A20
:100FBC00007BFFC3EB9AFCC3948250027C82757257
:100FCC00000572EC8572F0A4C3E5F0947D40F2222A
:100FDC00D27FF1A51205A01205A07A007B007C102F
:100FEC00120596E55C2AFA74003BFBDCF37C04C327
:100FFC00EB13FBEA13FADCF7FEC27F120FA5227586
:10100C007C00757D00E5EF20E6037520000520903F
:10101C003DFFE520146006901FFF146000930460F0
:10102C000375EF1653D9BF7581C043FF801205912C
:10103C0075EF0643B203E5B3240220E70DF521E575
:10104C00B120E0068521B343B101120E9D758038A5
:10105C0075A4C775F1FF75D4DF7590FF75A5007584
:0E106C00F20075D50075A0FF75A60075F300A3
:10107A0075D60075B0E475A71B75F4FF75E24112C9
:10108A000E9DE4F8F6D8FD756801120EB21215919C
:10109A0078988673753001C2AF1205AA1205BA1282
:1010AA0005A01205C11205A01205C81205A0121644
:1010BA00BA1205AA1205AA1205A5C2AF757C007557
:1010CA007D0078FA79FA308507D9FBD8F7021C0037
:1010DA00120F1E120F57120FA4120FA578988673BB
:1010EA00120E9D75881075890275C824759104754C
:1010FA00D84075A82275B80275E690759B80759DD3
:10110A000075D10E75BC5875BB0675BA1F75E88097
:10111A00120591D2AF12084975360053DACF207EF4
:10112A000343DA20307E0343DA1043DA01C2D8C21D
:10113A00711205AAD2617B037A0CE55B70077A0CFF
:10114A00DB030210C41205A02070030210C4C2708F
:10115A00E55CC3940240E1E52F541F855E5DF55EB0
:10116A00B55DD5DAD5C26153DACF207E0343DA20E2
:10117A00307E0343DA10C2D8C27178A2E67008D270
:10118A0074E52F54E0F52FC2757529001205A530B4
:10119A007409C3E529940A4002D2751205967802A9
:1011AA003074027800C3E55C9840F0C2AF1205BA09
:1011BA001205BA1205BAD2AF1205AA754C00788880
:1011CA00E6B4030241C4120596788CE6C394015032
:1011DA00030212C4E530C3940150030212C4757CA1
:1011EA00A5757DF1207435C3E55C94FF50030212A6
:1011FA00C4C2AF1205CFD2AF1205A5C3E55C9401F4
:10120A0050EFC2AF1205BA12059B1205BAD2AF123D
:10121A0005A5C3E55C94FF40E902173F7F05D27F2D
:10122A00120FA51205A5C2AFC27F120FA5AE5CC3ED
:10123A00E55C947FD2AF500241D4120591C2AF123D
:10124A0005CFD2AFDFD8120FDCC3EE94057897F63C
:10125A001205AA1216C27F0AD27F120FA51205A57D
:10126A00C2AFC27F120FA5AE5CC3E55C947FD2AF5A
:10127A0050E4120591C2AF1205BA12059B1205BAC3
:10128A00D2AFDFD4120FDCEE24037896F6F8799702
:10129A00E7C394824003985006E824827897F612AE
:1012AA0005AA1215DF1216F11205A5120FA5C3E53C
:1012BA005C94FF500221E802173F757C00757D009F
:1012CA00C3E55C954C4003855C4C1205A578017911
:1012DA0088E7B403027805C3E55C98400221C8C2D6
:1012EA00AF1205CF1205CF1205CFD2AF1205AA75DC
:1012FA003000E4F531F5320531E531F4703F05325D
:10130A00789AE67819146012783214600D787D1490
:10131A00600878FA146003753200C3E53298401DFC
:10132A00120E9D120591153275310078998673C295
:10133A00AF1205CFD2AF789886731205A512059B16
:10134A00E52A700530740201C47801207402780617
:10135A00C3E55C9840A17888E6C39403600312054C
:10136A00A5E52A70030210C4C2AF120E9DE4F5224D
:10137A00F523F524F525F526F567D2AF7885E6C37A
:10138A0033F565E4F544F545F546F547F548F57056
:10139A00F52CF52DF53775700875BB1E12059112DF
:1013AA00084D30EDFDA8BDA9BEE97001F88871129B
:1013BA00085175700875BB1E120F1EC2AF7561FF0A
:1013CA001208C7852261852262852263D2AF7522FF
:1013DA0001752401752501752601856069756A0103
:1013EA007888E6B40307C27D307602D27DD268D20D
:1013FA0069753300120DF6120E251208E71208EE6F
:10140A001208E71208EE1208E7120B6E1206B01263
:10141A000C63120CAA1208EE120B5D306E03120650
:10142A00B1206603120803306603120833120C63F4
:10143A00120CD91208EE120B6E306E031206ED1260
:10144A000C63120D501208EE120B5D306E03120778
:10145A004B120C63120D7F1208EE120B6E306E03E4
:0F146A001207A8120C63120DF61208EE12084DAD
:10147900120B5D120C63120E251208511208EE3080
:10148900692F856461856462856069756A01791867
:101499007A0CC3E53399400CC269D26A8A35756101
:1014A900FF0214BAC3E55C94014003021413021548
:1014B90048306A25206C22E535147006C26AD26B61
:1014C9008113F535C3E55C94014003021413788850
:1014D900E6C394036003021548753600788279A43F
:1014E900E760027803C3E55F985054307404E52A35
:1014F900604D7888E6B40317207D05207607A1188A
:10150900307602A118206C07D26C8564618152780B
:10151900F0306C058564617820C3E54198500281FB
:1015290013306C1BC26CC27D307602D27DD26A75D3
:10153900351285646181130536E55C6002A14B753E
:101549003600C2AF120E9D7887E6FE7602120F1E94
:101559007887EEF6E4F522F523F524F525F526F549
:1015690065752C00752D00D2AF1205A5120E9D7858
:10157900A4E66006D2B1D287D281307409C3E536B8
:101589009404400201C441FC901A0D7820121621DE
:10159900E520B45A0CA3121621E520B4A5030215BF
:1015A900BF757CA5757DF1120EB21215DF757C0031
:1015B900757D000215DE901A0378807B0A121621C8
:1015C900A308DBF9901A0F788C7B19121621A3084E
:1015D900DBF9901A2822C2AF121664121641901A2A
:1015E90000740E121626A37409121626A374151276
:1015F9001626901A0378807B0A121625A308DBF9B0
:10160900901A0F788C7B19121625A308DBF912168C
:1016190077121655901A2822E493F622E6438F0191
:10162900538FFDFFC3E583941C400122EF857CB7EE
:10163900857DB7F0538FFE22438F02438F01857C4E
:10164900B7857DB7901A0DF0538FFC22901A0D744F
:101659005AD126901A0E74A5D126227A3079D078DB
:1016690020901A40D121E520F709A3DAF7227A3030
:1016790079D0901A40E7D12609A3DAF922AB74A8E8
:1016890075BB01027984BB02027985BB03027986A5
:10169900BB04027992BB05027987BB060279A3BB19
:1016A9000702799CBB08027988BB09027989E8F7A6
:1016B900227C051205AADCFB22C2AF1205BA12056B
:1016C900C11205C81205CF12059B1205BA1205C130
:1016D9001205C81205CF12059B1205BA1205C112CF
:1016E90005C81205CFD2AF22C2AF1205CF1205C865
:1016F9001205C11205BA12059B1205CF1205C812AF
:1017090005C11205BA12059B1205CF1205C81205AB
:10171900C11205BAD2AF22AE74AF75C2AF1205BA03
:101729001205BA1205BA12059BDEF21205CF12058F
:101739009BDFF8D2AF22D1C2D1BAD1BA7574017583
:101749007501757600F1207C05AD5C1205AAC3ED23
:10175900955C70F5C3E55C9401400AC3E55C94FFB0
:10176900403202177BD186B1DFD1C2C2AF75EF1605
:10177900D1BADCD50576C3E5769403500280C6D18B
:10178900BA0575E5741490009F93F808C3E5759838
:10179900500280AED1BAD1BA0574C3E574940A5027
:0F17A90002809C120EB2B1DFC2AF75EF16D1BA3B
:0319FD0002100BCA
:101A00000E0915FFFFFFFF0304090301015AA50199
:101A1000FFFFFFFFFF03FFFFFF25D0FAFA04FF01DE
:091A2000007AFF0101000300FF40
:101A4000235475726E696779343041232020202039
:101A500023424C48454C4923463331302320202033
:101A60002020202020202020202020202020202076
:101C0000C2AFC2D353D9BF7581C043B20343FF8073
:101C1000752438752503B1DC7529A5752AF175E29F
:101C20004043F12053A4DF75D4FFD2857DFA7803B9
:101C300079E67C10752200752300901DE97B0675FE
:101C400024987525013085028145208508D8FBD967
:101C5000F9DCF781B7308508D8FBD9F9DCF781B713
:101C6000B19CE493A3C39A6004DDC381B7DBDBB10D
:101C70008E6002812E7B08E493FAA3B16FDBF87AC1
:101C800030B16F752200752300B18EEAFCEBFDC305
:101C9000ED94FE400EB18E8A278B28ED30E0048A49
:101CA000828B83B18E7AC270D8C3ED94FE601950D6
:101CB000CEBD002BEC600F7520007521FF7529004B
:101CC000752A000200008100A827A9280809D80465
:101CD000D90281DCB192EA89AAF281CE0D81A3C337
:101CE000ED94035053EDA2E092007AC5C3E58294CF
:101CF00000E583941C508A200010438F02438F011B
:101D00008529B7852AB7F0300029A827A92808090E
:101D1000438F01538FFDD804D902A133C3E58394C7
:101D20001C4003A3A11689AAE28529B7852AB7F02A
:101D3000A3A116538FFC817F7AC1BD030CE493A34A
:101D4000FAB153DCF8B14B817F8181AA22AB23B178
:101D50006FEBFAEA6222752608C3E52313F523E543
:101D60002213F52250066323A0632201D526EAB18F
:101D7000DCB1DC75260AEAF4200102D285300102CA
:101D8000C285B1DCC3134002C201D526EB22B19259
:101D9000EAFB208502A192308502A197752608AE44
:101DA00024AF25C3EF13FFEE13FEB1E0B1DCC3EAAD
:101DB000133085024480FA30E703632201C3E52330
:101DC00013F523E52213F52250066323A0632201B5
:101DD000D526D9E52265236523F52222AE24AF2539
:101DE0000E0FDEFEDFFCD20122424C48656C6934E6
:071DF000373164F310060116
:00000001FF
